:0300000002001DDE
:0300030002022FC7
:05000B007F00C28C32F1
:0300130002012FB8
:10001B00A33275B0FF7590FF3156758922758D012E
:10002B00758C0175880475A8CF75B804C28CC28E07
:10003B0075B0FF7590FFC2B57F007B00316CFD3151
:10004B00637F007B01316CFE7400145DFDBD000409
:10005B00EE4480FE783C793C7A007B007C007F008C
:10006B00D28EE968600411FF80F8E583B4FFF3904A
:10007B000000BC000280EB118680E711C674A01152
:10008B00D811E7740011D811E7740011D811E7EDFE
:10009B0011D811E711CF11EE11C674A011D811E7C9
:1000AB00740011D811E7740111D811E7EE11D811B2
:1000BB00E711CF11EE7C0090000022D2B7D2B5C26F
:1000CB00B7C2B522C2B7D2B5D2B7C2B5227A08C36E
:1000DB003392B700D2B500C2B5DAF422D2B7D2B59B
:1000EB00C2B52211C674A011D8D2B7D2B5A2B7C26D
:1000FB00B540F02208B88002783C11C674A011D824
:10010B0011E7ED11D811E7EE11D811E7E611D8116F
:10011B00E711CF0EBE00080DBD00047D007E8011DF
:10012B00EE7C0122758A0192D5F5F0EF1454F8702C
:10013B0012EBA2B413FBBF080A09B98002793CF792
:10014B00758A01D28C0FE5F0A2D53278057FFF7B43
:10015B00FFDBFEDFFAD8F6227FFF7BFFDBFEDFFA49
:10016B002211C674A011D811E7EF11D811E7EB11CA
:10017B00D811E711C674A111D811E77A087400C31E
:10018B00D2B5000030B701D3C2B50033DAF111E7B5
:10019B0011CF22309703C29722D29722309603C2F7
:1001AB009622D29622780A18B800FC2211C674A1A6
:1001BB0011D8D2B7D2B5A2B7C2B540F0227A64310A
:1001CB00B01ABA00FA2220B30531C830B3FB7C0059
:1001DB0051047A08C313500651110C0201EB510460
:1001EB001ABA00F0C3EC13500551040201FB511174
:1001FB0051117C3C31B0DCFC22D2B3C2B431B0C261
:10020B00B331B0D2B322D2B3D2B431B0C2B331B066
:10021B00D2B32290035093F5F031D174F031D1E584
:10022B00F031D12275A80075880431561186EDFF87
:10023B00EEFB740054F0C4511E7400540F511EEDAC
:10024B0054F0C4511EED540F511EEE54F0C4511E08
:10025B00EE540F511E316CF954F0C4511EE9540F7A
:10026B00511E30B2131BBBFF011FBF00E8BB7FE564
:10027B007BFF7F001F0202603156783C793C7A008D
:10028B007B007C007F0075880475A8CF75B804D2FD
:02029B008E32A1
:1003500045161E26252E363D3E461C322123242BD3
:01036000227A
:00000001FF
